:107E000001C0ABC0112484B7882361F0982F9A7009
:107E1000923041F081FF02C097EF94BF282E80E09E
:107E2000BFD0EEC085E08093810082E08093C000E7
:107E300088E18093C10089E18093C40086E080934B
:107E4000C2008EE0ADD0259A84E028E13EEF91E0BB
:107E5000309385002093840096BBB09BFECF1D9A83
:107E6000A8954091C00047FD02C0815089F78CD091
:107E7000813461F489D0182F99D01238E9F0113883
:107E800011F488E001C083E078D064C0823411F43A
:107E900084E103C0853419F485E090D05BC085355A
:107EA00039F472D0C82F70D0D82FCC0FDD1F51C03D
:107EB000863521F484E082D080E0E6CF843661F517
:107EC00063D062D0D82E60D0F82E00E011E05CD0F4
:107ED000F80181938F01DE12FACF68D0F5E4FF122A
:107EE00001C0FFCF40E050E063E0CE0136D07E011C
:107EF00000E011E0F801419151918F0161E0C7016B
:107F00002CD0F2E0EF0EF11CD012F4CF40E050E0A4
:107F100065E0CE0122D01EC0843771F435D034D054
:107F2000F82E32D043D08E01F80185918F0125D0F3
:107F3000FA94F110F9CF0EC0853739F437D08EE1BD
:107F40001CD085E91AD086E19FCF813511F488E0F5
:107F500027D02CD080E111D08ACFFC010A0167BF65
:107F6000E895112407B600FCFDCF667029F0452B7B
:107F700019F481E187BFE89508959091C00095FFBD
:107F8000FCCF8093C60008958091C00087FFFCCF8E
:107F90008091C00084FD01C0A8958091C60008951D
:107FA000E0E6F0E098E1908380830895EDDF803291
:107FB00019F088E0F5DFFFCF84E1DFCFCF93C82F42
:0A7FC000E3DFC150E9F7CF91F1CFE4
:027FFE00000879
:0400000300007E007B
:00000001FF
